:100000000C9474010C9491010C9491010C94910145
:100010000C9491010C9491010C9491010C94910118
:100020000C9491010C9491010C9491010C94910108
:100030000C9491010C9491010C9491010C949101F8
:100040000C9491010C9491010C9491010C949101E8
:100050000C9491010C94D7060C9491010C9491018D
:100060000C9491010C949101808183848687898A04
:100070008C8E8F9192949597989A9B9D9EA0A2A307
:10008000A5A6A7A9AAACADAFB0B2B3B5B6B7B9BA79
:10009000BCBDBEC0C1C2C4C5C6C8C9CACBCDCECF07
:1000A000D0D2D3D4D5D6D7D9DADBDCDDDEDFE0E1C0
:1000B000E2E3E4E5E6E7E8E9EAEAEBECEDEEEEEFB1
:1000C000F0F1F1F2F3F3F4F5F5F6F6F7F8F8F9F9E3
:1000D000FAFAFAFBFBFCFCFCFDFDFDFDFEFEFEFE5C
:1000E000FEFFFFFFFFFFFFFF0000891112239B327D
:1000F0002446AD573665BF74488CC19D5AAFD3BEF8
:100100006CCAE5DB7EE9F7F88110080193331A2207
:10011000A5562C47B7753E64C99C408DDBBF52AED7
:10012000EDDA64CBFFF976E802218B3010029913E7
:100130002667AF763444BD554AADC3BC588ED19FB7
:100140006EEBE7FA7CC8F5D983310A2091121803C7
:10015000A7772E66B5543C45CBBD42ACD99E508F97
:10016000EFFB66EAFDD874C904428D5316619F7097
:100170002004A9153227BB364CCEC5DF5EEDD7FC77
:100180006888E1997AABF3BA85520C4397711E6087
:10019000A1142805B3373A26CDDE44CFDFFD56EC57
:1001A000E9986089FBBB72AA06638F7214409D5167
:1001B0002225AB343006B9174EEFC7FE5CCCD5DD37
:1001C0006AA9E3B8788AF19B87730E6295501C4147
:1001D000A3352A24B1163807CFFF46EEDDDC54CD17
:1001E000EBB962A8F99A708B088481951AA793B627
:1001F0002CC2A5D33EE1B7F04008C919522BDB3A17
:10020000644EED5F766DFF7C899400859BB712A6E6
:10021000ADD224C3BFF136E0C1184809D33B5A2AF6
:10022000E55E6C4FF77D7E6C0AA583B418869197C6
:100230002EE3A7F23CC0B5D14229CB38500AD91BD6
:10024000666FEF7E744CFD5D8BB502A499961087A6
:10025000AFF326E2BDD034C1C3394A28D11A580BB6
:10026000E77F6E6EF55C7C4D0CC685D71EE597F476
:100270002880A1913AA3B3B2444ACD5B5669DF7896
:10028000600CE91D722FFB3E8DD604C79FF516E466
:10029000A9902081BBB332A2C55A4C4BD7795E6876
:1002A000E11C680DF33F7A2E0EE787F61CC495D546
:1002B0002AA1A3B03882B193466BCF7A5448DD5956
:1002C000622DEB3C700EF91F8FF706E69DD414C526
:1002D000ABB122A0B9923083C77B4E6AD5585C4936
:1002E000E33D6A2CF11E780F11241FBECFEFD8E03A
:1002F000DEBFCDBF11E0A0E0B1E0E0EDFAE202C068
:1003000005900D92A231B107D9F718E0A2E1B1E052
:1003100001C01D92A039B107E1F70E94FD130C94B2
:1003200066150C9400000C945C12789488E997E0B0
:100330000E9413038FEF9FEF9093750880937408CA
:10034000909377088093760823E931E048E957E0F5
:1003500064E778E08AE394E00E94C80786E698E0C4
:100360000E94D10186E698E090938D0880938C08D6
:1003700090938B0880938A08AC0168E977E08AE360
:1003800094E00C944F129091C00095FFFCCF8093A5
:10039000C60008958091C00087FFFCCF8091C60001
:1003A0000895CF93DF93CDB7DEB72E970FB6F894AD
:1003B000DEBF0FBECDBFDC019EE0FD01892F119293
:1003C0008A95E9F71092C50087E68093C400E0ECB7
:1003D000F0E080818D7F808386E08093C20088E199
:1003E0008093C1009E012F5F3F4FF90111929A95B2
:1003F000E9F783E08C8383EC91E09A8789878AEC24
:1004000091E09C878B878EE0F90101900D928A958F
:10041000E1F72E960FB6F894DEBF0FBECDBFDF9189
:10042000CF910895811106C08091C000881F882750
:10043000881F089580E008958091C00087FF03C061
:100440008091C60008958FEF0895E0917808F091AB
:1004500079084FB7F894EB58FF4F24813581868196
:1004600097814FBF28173907E1F0E0917808F091A4
:1004700079082FB7F894EB58FF4FA481B58182819A
:100480009381A817B90719F48081918104C0A481D0
:10049000B581CD010196958384838C912FBF90E027
:1004A00008958FEF9FEF08950F931F93CF93DF93DE
:1004B000182FC0917808D0917908FE01E959FF4FB3
:1004C0008081811124C080E490E09E8F8D8F1C8EEE
:1004D0001B8E1A8E01E00083299A20910901309128
:1004E0000A0140910B0150910C01A0EBB4E00E9475
:1004F0001C146056704F8F4F9F4F20E43FE140E047
:1005000050E00E944F143B8B2A8B009313010FB7CE
:10051000F894209105013091060140910701509116
:100520000801A0EBB4E00E941C146056704F8F4F7E
:100530009F4F20E43FE140E050E00E944F143D8B8C
:100540002C8B0FBFE0917808F09179085FB7F89491
:1005500023A134A1878D90A12817390739F425A14B
:1005600036A181A192A12817390761F025A136A1F2
:1005700083A194A1019741E02817390709F040E0D1
:10058000842F01C081E05FBF80FDDCCFE09178085F
:10059000F09179084FB7F894A5A1B6A11C9325A1B5
:1005A00036A181A192A12817390719F4878D90A14E
:1005B00003C085A196A1019696A385A34FBFDF91A5
:1005C000CF911F910F91089581E0809312010895BA
:1005D00081E0809312011092800089E18093810074
:1005E00081E896E0909387008093860080911201C5
:1005F000882321F080E480937C0002C010927C006C
:100600003898409880917E00816080937E0087E0DA
:1006100080937B008CEE80937A008AB1886F8AB9D0
:10062000219A229A08950F931F93CF93DF93CDB70A
:10063000DEB72E970FB6F894DEBF0FBECDBF8C018C
:100640008AECD8011D928A95E9F7109379080093F6
:10065000780880E490E0F801968F858FC801805972
:100660009F4FE859FF4F91838083978386839583BB
:100670008483C8018C589F4F93838283C801835819
:100680009F4FD801AB58BF4F11969C938E931796EE
:100690009C938E93169715969C938E931497C801EE
:1006A00084549F4F13969C938E931297C8018796FC
:1006B000D80190969C938E935F9796969C938E9379
:1006C000959794969C938E939397C8018A599F4FC0
:1006D00092969C938E93919784E090E0A681B78147
:1006E0001C9246815781228133814217530719F4A6
:1006F0002081318104C0268137812F5F3F4F3783AE
:1007000026830197009751F70E94E8022EE0FE0130
:100710003196DF01822F1D928A95E9F783E08C8361
:1007200084E592E09A87898785E292E09C878B87AF
:10073000D80101900D922A95E1F72E960FB6F89404
:10074000DEBF0FBECDBFDF91CF911F910F910895F6
:100750000F931F93CF93DF938B01E0917808F09173
:10076000790825A136A134A323A3EC01080F191F92
:10077000C017D10721F089910E945402F9CFDF916F
:10078000CF911F910F910895DC0156968C91569749
:100790008111E9C058968C91589781119FC093960A
:1007A0002D913C91949795968D919C9196972817B1
:1007B000390739F454968D919C915597892B09F4FA
:1007C0005CC059968C915997811103C05A961C921E
:1007D0005A9781E059968C93599752968D919C9196
:1007E0005397009789F593962D913C919497959600
:1007F0008D919C9196972817390751F454968D91B5
:100800009C915597019755969C938E93549721C030
:100810009396ED91FC91949791968D919C919297DE
:10082000E817F90729F45F968D919C91909706C07F
:100830009396ED91FC919497CF01019694969C9399
:100840008E939397808106C0019753969C938E93C5
:1008500052978EE757968C93579757968C91579748
:100860008B3191F593962D913C91949795968D911E
:100870009C9196972817390741F410921301A959B2
:10088000BF4F1C92299880E008959396ED91FC91BA
:10089000949791968D919C919297E817F90729F476
:1008A0005F968D919C91909706C09396ED91FC91E7
:1008B0009497CF01019694969C938E939397808101
:1008C00057968C93579706C08E57823018F45996D6
:1008D0001C92599781E058968C93589759962C9171
:1008E00059975D968D919C915E972223A9F05A9617
:1008F0002C915A97253080F05A961C925A97803442
:10090000910519F485E790E002C080E490E05E96DE
:100910009C938E935D9723C058963C915897579619
:100920002C915797232341F05A968C915A978F5FB9
:100930005A968C935A970FC05A961C925A978034A5
:10094000910519F485E790E002C080E490E05E969E
:100950009C938E935D97330F58963C93589788E0FD
:1009600056968C9356975D96ED91FC915E975B96AB
:100970008D919C915C97E80FF91F9F0131705C96F7
:100980003C932E935B9756968C9156978150569632
:100990008C93FF27E038F10530F08FEF90E0AC0149
:1009A0004E1B5F0BFA01E859FF4F84912F3F310531
:1009B00011F008F080950895EF92FF920F931F9326
:1009C000CF93DF93FC018C0101541F4FD8014D914F
:1009D0005C91DC01A354BF4F4D935C93DC01A8599B
:1009E000BF4F14968D919C91159712962D913C9125
:1009F00013978217930721F42D913C91119707C00B
:100A000014968D919C9115979C012F5F3F4F1596E1
:100A10003C932E931497EC0188818602C001112427
:100A20009595879595958795E801998388837F01AA
:100A3000D3ECED0EF11CE701288139818F010F53B2
:100A40001F4FE80139832883840F951F359527951B
:100A5000820F931FE70199838883AF014B535F4F48
:100A600021E0181619060CF020E0EA018881880FB1
:100A7000822B888316968D919C911797EC01688341
:100A800016962D913C91179712968D919C911397E4
:100A90002817390721F48D919C91119705C016965E
:100AA0008D919C911797019617969C938E9316970C
:100AB000DA019C91892F8695869589278370DF01BD
:100AC000AA53BF4F833039F48C91803214F48F5F76
:100AD00001C081508C938C91885F8C9380340CF48E
:100AE0005FC18F738C93DF01A953BF4F8C91880F27
:100AF00097702BEF290F233010F0933009F48160A9
:100B00008C939C91892F86958927809581709685F5
:100B1000990F892B86878E3709F04EC0DF01AB58BD
:100B2000BF4F14962D913C9115978D919C911197E3
:100B30002817390759F416962D913C91179712965C
:100B40008D919C9113972817390781F016962D9156
:100B50003C91179714968D919C911597019741E0C0
:100B60002817390709F040E0842F01C081E080FD9B
:100B7000DCC01696CD91DC9117978EE78883169688
:100B80002D913C91179712968D919C911397281750
:100B9000390721F48D919C91119705C016968D917E
:100BA0009C911797019617969C938E93169781E0C8
:100BB000818B2A9A41E0BCC0982F9F779F3719F408
:100BC000118A2A98EDC09189992309F4E9C0982FD8
:100BD0009F739E3309F4E4C080FF03C0808980685E
:100BE000808B87858F5F87879089883008F4A5C0C0
:100BF000DF01AB58BF4F82E8890F823018F09B317C
:100C000009F04BC014962D913C9115978D919C91B4
:100C100011972817390759F416962D913C9117977B
:100C200012968D919C9113972817390781F016968B
:100C30002D913C91179714968D919C911597019742
:100C400041E02817390709F040E0842F01C081E016
:100C500080FD1FC01696CD91DC9117978BE188839C
:100C600016962D913C91179712968D919C91139702
:100C70002817390721F48D919C91119705C016967C
:100C80008D919C911797019617969C938E9316972A
:100C900004C0118A2A9840E001C041E014962D91C9
:100CA0003C9115978D919C9111972817390759F40C
:100CB00016962D913C91179712968D919C911397B2
:100CC0002817390781F016962D913C9117971496A5
:100CD0008D919C911597019751E02817390709F0DC
:100CE00050E0852F01C081E080FD1FC080891696ED
:100CF000CD91DC911797888316962D913C9117978B
:100D000012968D919C9113972817390721F48D9194
:100D10009C91119705C016968D919C9117970196FD
:100D200017969C938E93169703C0118A2A9840E0D9
:100D3000108A1786442321F033C09695908B30C0DB
:100D4000DF01A853BF4F8D919C911197816011963F
:100D50009C938E93EB58FF4F248135818081918144
:100D60002817390739F42681378182819381281722
:100D7000390761F02681378184819581019741E0AF
:100D80002817390709F040E0842F01C081E080FF77
:100D900007C0868197819583848311961C921E9249
:100DA000DF91CF911F910F91FF90EF9008951F92C7
:100DB0000F920FB60F9211242F933F934F935F938F
:100DC0006F937F938F939F93AF93BF93EF93FF9313
:100DD00080E286BB60917800709179007695679586
:100DE00076956795605880917808909179080E946F
:100DF000DC0480911301882349F080917808909158
:100E000079080E94C403807F886001C080E88BB9A4
:100E10008091620890916308A0916408B091650880
:100E20000196A11DB11D8093620890936308A09361
:100E30006408B0936508FF91EF91BF91AF919F91C6
:100E40008F917F916F915F914F913F912F910F9073
:100E50000FBE0F901F9018951F93CF93DF93EC0157
:100E6000162F82E8860F823010F06B3131F46881E2
:100E700079818BE190E00E940D1568817981812F45
:100E800090E0DF91CF911F910C940D150F931F935C
:100E9000CF93DF938C010F5B1C4FD8012D913C91B8
:100EA000232B49F1EC01498550E0DC01AC5CBC4FDF
:100EB0002D913C9111972C503109241B350B119623
:100EC0003C932E93FC012D913C911197BF01681B1F
:100ED000790B6217730738F49F01240F351FE9015E
:100EE0002A852193F0CFD801ED91FC91DF91CF912C
:100EF0001F910F910994DF91CF911F910F91089548
:100F0000AF92BF92CF92DF92EF92FF920F931F9317
:100F1000CF93DF935B016A017C0126ECE21A2CEF90
:100F2000F20A2FEF3FEFF701318320838C01005D40
:100F30001C4FF801608171818EE790E00E940D15D1
:100F4000E501CA0CDB1CCC15DD0529F06991C8014F
:100F50000E942C07F8CFF7016081C1816095C8011C
:100F60000E942C076C2F6095C8010E942C07F80185
:100F7000608171818EE790E0DF91CF911F910F9199
:100F8000FF90EF90DF90CF90BF90AF900C940D1535
:100F9000CF93DF93EEE5F3E0DC01EF011D922197A3
:100FA000E9F7FC01E05DFC4F51834083FC01EF5BFE
:100FB000FC4F31832083FC01EE5CFC4F7183608326
:100FC000FC01E65CFC4F2FEF3FEF31832083FC01F7
:100FD000E85CFC4F3183208330937B0820937A08B0
:100FE00030937D0820937C08DF91CF9108952F9254
:100FF0003F924F925F926F927F928F929F92AF92A9
:10100000BF92CF92DF92EF92FF920F931F93CF93F5
:10101000DF93CDB7DEB728970FB6F894DEBF0FBECB
:10102000CDBF282F21702B8383FB442440F8512C03
:1010300081FBAA27A0F9B0E0A425B52584FB3327BE
:1010400030F93F83188686FB772770F979831A82F7
:1010500082FB662460F8712C85FB222420F8312C59
:101060008078E82FF0E0EE0FEF2FEE1FFF0BFE83EE
:10107000ED83F62FF170FC8363FB882480F8912CBC
:1010800061FB222720F930E02825392564FB44271D
:1010900040F950E066FB002700F910E062FBCC2429
:1010A000C0F8D12C65FBEE24E0F8F12C607870E0FC
:1010B000660F672F661F770B402751275A01AE2412
:1010C000BF24A626B726C9018C259D2586279727EC
:1010D0008295880F880F807C60E8A69E8019112475
:1010E000EF81F88569817A81E627F727F887EF8312
:1010F0009E2F91707B8197273A2F31709327890F0C
:10110000A625B7259D81A927E4E0AE9F800D112477
:10111000EF81F885E225F3256D817E81E627F727AB
:1011200078E0E79F800D112441709C814927217050
:101130004227E0E14E9F800D112496012E253F2588
:10114000922F9170FC819F27082519250170902707
:1011500020E2929F800D1124930122253325922FA6
:1011600091703B81932729813A812425352521706F
:101170009227990F890F28960FB6F894DEBF0FBEFD
:10118000CDBFDF91CF911F910F91FF90EF90DF9036
:10119000CF90BF90AF909F908F907F906F905F9017
:1011A0004F903F902F9008952F923F924F925F92D1
:1011B0006F927F928F929F92AF92BF92CF92DF9267
:1011C000EF92FF920F931F93CF93DF9300D000D045
:1011D000CDB7DEB74C01FC01EB5BFC4F8081D40145
:1011E000A80FB11DAA5BBC4F6C938F5F80838C30BE
:1011F00009F09BC3C401805D9C4F9C838B83F401E9
:10120000EA5BFC4FFA83E9838081807891E0803843
:1012100009F090E09795992797955401F9EBAF1A4B
:10122000FCEFBF0AF5018081807841E0803809F049
:1012300040E0F0E44F9F900D1124492F640120EB12
:10124000C21A2CEFD20AF6018081807891E08038B2
:1012500009F090E0490F7401F7EBEF1AFCEFFF0A79
:10126000F7018081807891E0803809F090E0F0E229
:101270009F9F400D11248401065B1C4FF801808163
:10128000807891E0803809F090E0F0E19F9F400D78
:101290001124340124EB621A2CEF720AF3018081CD
:1012A000807891E0803809F090E0F8E09F9F400D51
:1012B0001124240123EB421A2CEF520AF2019081EF
:1012C000907881E0903809F080E0880F880F840FD3
:1012D0001401F1EB2F1AFCEF3F0AF1019081907895
:1012E00061E0903809F060E0660F680F8B819C81A7
:1012F0000E942C07E981FA81908181E096FF80E0CD
:10130000879588278795F501408191E046FF90E019
:10131000F0E49F9F800D1124982FF601408181E019
:1013200046FF80E0980FF701408181E046FF80E0B2
:10133000F0E28F9F900D1124F801408181E046FF7B
:1013400080E0F0E18F9F900D1124F301408181E056
:1013500046FF80E0F8E08F9F900D1124F20140815C
:1013600081E046FF80E0880F880F890FF1019081AE
:1013700061E096FF60E0660F680F8B819C810E94A0
:101380002C07E981FA81908181E095FF80E08795C3
:1013900088278795F501408191E045FF90E0F0E4D2
:1013A0009F9F800D1124982FF601408181E045FF19
:1013B00080E0980FF701408181E045FF80E0F0E296
:1013C0008F9F900D1124F801408181E045FF80E05E
:1013D000F0E18F9F900D1124F301408181E045FFE2
:1013E00080E0F8E08F9F900D1124F201408181E0B0
:1013F00045FF80E0880F880F890FF101908161E03F
:1014000095FF60E0660F680F8B819C810E942C071E
:10141000E981FA81908181E094FF80E087958827B7
:101420008795F501408191E044FF90E0F0E49F9FB3
:10143000800D1124982FF601408181E044FF80E067
:10144000980FF701408181E044FF80E0F0E28F9F38
:10145000900D1124F801408181E044FF80E0F0E12B
:101460008F9F900D1124F301408181E044FF80E0C3
:10147000F8E08F9F900D1124F201408181E044FF3C
:1014800080E0880F880F890FF101908161E094FF5F
:1014900060E0660F680F8B819C810E942C07C4015D
:1014A0008A5B9C4F9A838983FC01908181E093FF42
:1014B00080E08795882787955401F9EBAF1AFCEFF8
:1014C000BF0AF501408191E043FF90E0F0E49F9F67
:1014D000800D1124982F640120EBC21A2CEFD20A40
:1014E000F601408181E043FF80E0980F7401F7EB43
:1014F000EF1AFCEFFF0AF701408181E043FF80E033
:10150000F0E28F9F900D11248401065B1C4FF801BF
:10151000408181E043FF80E0F0E18F9F900D112436
:10152000340124EB621A2CEF720AF301408181E04E
:1015300043FF80E0F8E08F9F900D1124240123EBFE
:10154000421A2CEF520AF201408181E043FF80E011
:10155000880F880F890F1401F1EB2F1AFCEF3F0A57
:10156000F101908161E093FF60E0660F680F8B816D
:101570009C810E942C07E981FA81908181E092FF91
:1015800080E0879588278795F501408191E042FFAB
:1015900090E0F0E49F9F800D1124982FF601408188
:1015A00081E042FF80E0980FF701408181E042FF37
:1015B00080E0F0E28F9F900D1124F801408181E0DE
:1015C00042FF80E0F0E18F9F900D1124F3014081F4
:1015D00081E042FF80E0F8E08F9F900D1124F2013E
:1015E000408181E042FF80E0880F880F890FF10180
:1015F000908161E092FF60E0660F680F8B819C81B3
:101600000E942C07E981FA81908181E091FF80E0BE
:10161000879588278795F501408191E041FF90E00B
:10162000F0E49F9F800D1124982FF601408181E006
:1016300041FF80E0980FF701408181E041FF80E0A9
:10164000F0E28F9F900D1124F801408181E041FF6D
:1016500080E0F0E18F9F900D1124F301408181E043
:1016600041FF80E0F8E08F9F900D1124F20140814E
:1016700081E041FF80E0880F880F890FF1019081A0
:1016800061E091FF60E0660F680F8B819C810E9492
:101690002C07E981FA818081F50160816170629592
:1016A000660F660F607CF0E88F9F60191124F601C9
:1016B00080818170680FF70180818170F0E28F9FD7
:1016C000600D1124F80180818170F0E18F9F600D21
:1016D0001124F30180818170F8E08F9F600D112447
:1016E000F20180818170880F880F680FF10180817D
:1016F0008170880F680F8B819C810E942C07540198
:10170000F8EBAF1AFCEFBF0AF50170816401F5EB4D
:10171000CF1AFCEFDF0AF60150817401F2EBEF1AE9
:10172000FCEFFF0AF701408184010F5A1C4FF801BA
:101730009081672F607881E0603809F080E08795BC
:101740008827879561E073FF60E0F0E46F9F800D6C
:101750001124682F81E093FF80E0680F81E0752FEE
:101760007078703809F080E020E2829F600D1124CB
:1017700081E053FF80E0562FE0E18E9F500D112451
:1017800081E0642F6078603809F080E0F8E08F9F96
:10179000500D112481E043FF80E0880F880F850FF2
:1017A000907861E0903809F060E0660F680F8B81F7
:1017B0009C810E942C07F5017081F6015081F70190
:1017C0004081F801908181E076FF80E0879588274D
:1017D000879561E072FF60E0F0E46F9F800D112457
:1017E000682F81E092FF80E0680F81E056FF80E083
:1017F00020E2829F600D112481E052FF80E0562F8D
:10180000E0E18E9F500D112481E046FF80E0F8E07A
:101810008F9F500D112481E042FF80E0880F880FD8
:10182000850F61E096FF60E0660F680F8B819C81F9
:101830000E942C07F5017081F6015081F70140816B
:10184000F801908181E075FF80E087958827879572
:1018500061E071FF60E0F0E46F9F800D1124682F5C
:1018600081E091FF80E0680F81E055FF80E020E299
:10187000829F600D112481E051FF80E0562FE0E14E
:101880008E9F500D112481E045FF80E0F8E08F9F8E
:10189000500D112481E041FF80E0880F880F850FF3
:1018A00061E095FF60E0660F680F8B819C810E946C
:1018B0002C07F5017081F6016081F7015081F80174
:1018C0004081972F9170862F81708295807FF0E400
:1018D0009F9F800D1124942F9170890F952F9170E7
:1018E000990F990F890F91E074FF90E020E8929F83
:1018F0008019112491E064FF90E0E0E29E9F800D4A
:10190000112491E054FF90E0F8E09F9F800D112496
:1019100061E044FF60E0660F680F8B819C810E944C
:101920002C07F401EB5BFC4F10820F900F900F908F
:101930000F90DF91CF911F910F91FF90EF90DF906B
:10194000CF90BF90AF909F908F907F906F905F905F
:101950004F903F902F9008951F93CF93DF93EC010A
:10196000162F0E94D408DE01A65CBC4F2D913C913D
:101970001197F901E127FF27EE0FFF1FE851FF4FF5
:1019800085919491232F3327822793278D939C93BE
:1019900080911501882349F0612F809114010E94E4
:1019A000F707682FCE010E94D4081093140180918C
:1019B000150191E0892780931501DF91CF911F9147
:1019C00008950F931F93CF93DF93EC018B01FB01DD
:1019D00061810E94AC0CF8016081CE010E94AC0CC8
:1019E000F8016381CE010E94AC0CF8016281CE0146
:1019F000DF91CF911F910F910C94AC0C6F927F925D
:101A00008F929F92AF92BF92CF92DF92EF92FF920E
:101A10000F931F93CF93DF93CDB7DEB72A970FB6FF
:101A2000F894DEBF0FBECDBF8C013A014901FC0125
:101A3000EB5BFC4F10826C0186ECC81A8CEFD80A65
:101A40008FEF9FEFF60191838083CE0101967C0199
:101A50008AE0F70111928A95E9F7F801EE5CFC4FF4
:101A60000190F081E02D808191819A838983828128
:101A700093819C838B83FB01808191819E838D83E5
:101A80008281938198878F838CE0820F877011F415
:101A90001A8603C098E0981B9A875801F0EDAF1A98
:101AA000FCEFBF0AF501608171818EE790E00E9432
:101AB0000D15B701C8010E94E10CBE016B5F7F4F9D
:101AC000C8010E94E10C6985C8010E94AC0C6A85BE
:101AD000C8010E94AC0C8A859FEF980F9A878823D3
:101AE00011F060E0F5CF7301860C971CE814F9043F
:101AF00039F0F70161917F01C8010E94AC0CF6CF6B
:101B0000F6016081F1806095C8010E94AC0C6F2DD8
:101B10006095C8010E94AC0CF501608171818EE76F
:101B200090E00E940D152A960FB6F894DEBF0FBE06
:101B3000CDBFDF91CF911F910F91FF90EF90DF907C
:101B4000CF90BF90AF909F908F907F906F900895AF
:101B50009A01AB016AE778E00C94FE0C4F925F9219
:101B60007F928F929F92AF92BF92CF92DF92EF922D
:101B7000FF920F931F93CF93DF939C012E5A3C4FFC
:101B8000F901D080EC01CD5ADC4FC880DC01AC5AA1
:101B9000BC4FEC902C01FBEA4F1AFCEF5F0AF201FC
:101BA000F080AC014A5A5C4FFA010081AC01495AFD
:101BB0005C4FFA011081AC01485A5C4FFA01708108
:101BC000AC01475A5C4FFA01B080AC01465A5C4FF9
:101BD000FA016081AC01455A5C4FFA01A080AC016A
:101BE000445A5C4FFA019080AC01435A5C4FFA01B1
:101BF0004081FD2DF07851E0E0E8FE1350E0752EB5
:101C000077947724779451E0FC2DF078E0E8FE1388
:101C100050E0F0E45F9F700C112451E0EB2DE07870
:101C2000F0E8EF1350E0750E51E0EE2DE078F0E8AB
:101C3000EF1350E0E0E25E9F700C112451E0FF2DA5
:101C4000F078E0E8FE1350E0F0E15F9F700C1124A3
:101C500051E0E02FE078F0E8EF1350E0E8E05E9F1D
:101C6000700C112451E0F12FF078E0E8FE1350E001
:101C7000852E880C880C870C51E0F72FF078E0E86F
:101C8000FE1350E0550F580DF901508321E0D6FEA8
:101C900020E027952227279531E0C6FE30E0F0E4CA
:101CA0003F9F200D1124322F21E0B6FE20E0320F9D
:101CB00021E0E6FE20E050E2259F300D112421E0D6
:101CC000F6FE20E0E0E12E9F300D112421E006FF1A
:101CD00020E0F8E02F9F300D1124232F31E016FF74
:101CE00030E0330F330F320F21E076FF20E0220F78
:101CF000230F288321E0362F3078303809F020E098
:101D000027952227279531E05A2D5078503809F031
:101D100030E050E4359F200D1124322F21E046FFA2
:101D200020E0320F21E0592D5078503809F020E0A2
:101D3000E0E22E9F300D112421E0542F50785038CE
:101D400009F020E0F0E12F9F300D112421E066FF23
:101D500020E058E0259F300D1124232F31E0A6FE0E
:101D600030E0330F330F320F21E096FE20E0220FD8
:101D7000230F2C9321E0D5FE20E0279522272795DD
:101D800031E0C5FE30E0E0E43E9F200D1124322F0B
:101D900021E0B5FE20E0320F21E0E5FE20E0F0E298
:101DA0002F9F300D112421E0F5FE20E050E1259F0A
:101DB000300D112421E005FF20E0E8E02E9F300DDA
:101DC0001124232F31E015FF30E0330F330F320F92
:101DD00021E075FF20E0220F230FF2012083FC0198
:101DE000EA5AFC4F21E0D4FE20E0279522272795D0
:101DF00031E0C4FE30E050E4359F200D1124322F35
:101E000021E0B4FE20E0320F21E0E4FE20E050E2C9
:101E1000259F300D112421E0F4FE20E050E1259FA4
:101E2000300D112421E004FF20E058E0259F300D03
:101E30001124232F31E014FF30E0330F330F320F22
:101E400021E074FF20E0220F230F2083FC01E95AD8
:101E5000FC4F21E065FF20E027952227279531E000
:101E6000A5FE30E050E4359F200D1124322F21E0F3
:101E700044FF20E0320F21E095FE20E050E2259F54
:101E8000300D112421E045FF20E050E1259F300D69
:101E9000112421E064FF20E058E0259F300D11243B
:101EA000232F31E0A4FE30E0330F330F320F21E057
:101EB00094FE20E0220F230F2083FC01E85AFC4F00
:101EC00021E0D3FE20E027952227279531E0C3FEAD
:101ED00030E050E4359F200D1124322F21E0B3FE75
:101EE00020E0320F21E0E3FE20E050E2259F300D9C
:101EF000112421E0F3FE20E050E1259F300D112454
:101F000021E003FF20E058E0259F300D1124232F0E
:101F100031E013FF30E0330F330F320F21E073FF56
:101F200020E0220F230F2083FC01E75AFC4F21E021
:101F3000D2FE20E027952227279531E0C2FE30E02F
:101F400050E4359F200D1124322F21E0B2FE20E015
:101F5000320F21E0E2FE20E050E2259F300D1124F7
:101F600021E0F2FE20E050E1259F300D112421E018
:101F700002FF20E058E0259F300D1124232F31E08F
:101F800012FF30E0330F330F320F21E072FF20E0F9
:101F9000220F230F2083FC01E65AFC4F21E063FF50
:101FA00020E027952227279531E0A3FE30E050E47A
:101FB000359F200D1124322F21E042FF20E0320F07
:101FC00021E093FE20E050E2259F300D112421E016
:101FD00043FF20E050E1259F300D112421E062FFF6
:101FE00020E058E0259F300D1124232F31E0A2FE80
:101FF00030E0330F330F320F21E092FE20E0220F4A
:10200000230F2083FC01E55AFC4F21E0D1FE20E0A4
:1020100027952227279531E0C1FE30E050E4359F17
:10202000200D1124322F21E0B1FE20E0320F21E0FB
:10203000E1FE20E050E2259F300D112421E0F1FE69
:1020400020E050E1259F300D112421E001FF20E028
:1020500058E0259F300D1124232F31E011FF30E08F
:10206000330F330F320F21E071FF20E0220F230FD7
:102070002083FC01E45AFC4F2C2D21702295220F65
:10208000220F207C30E8D39E201911243B2D317083
:10209000230F3E2D317050E2359F200D11243F2D2E
:1020A000317050E1359F200D1124017038E0039FFD
:1020B000200D11241170110F110F210F7170770F66
:1020C000270F2083FC01E35AFC4F362F31702A2D55
:1020D0002170220F220F58E0359F200D1124342F3C
:1020E0003170230F392D3170330F230F31E061FF31
:1020F00030E080E8389F2019112431E0A1FE30E063
:1021000050E4359F200D112431E091FE30E080E253
:10211000389F200D112431E041FF30E040E1349F31
:10212000200D11242083DF91CF911F910F91FF90FB
:10213000EF90DF90CF90BF90AF909F908F907F9067
:102140005F904F9008952F923F924F925F926F92BF
:102150007F928F929F92AF92BF92CF92DF92EF9237
:10216000FF920F931F93CF93DF93CDB7DEB72997DD
:102170000FB6F894DEBF0FBECDBF8C011C012DEB56
:10218000221A2CEF320A6C014CEBC41A4CEFD40A21
:102190007C018CECE81A8CEFF80AD801A85CBC4FE3
:1021A0002D01F801E35CFC4FFC83EB83C801845CE8
:1021B0009C4F9E838D83F801E05DFC4F808191816F
:1021C0000E94CF149C012F3F9FEF390709F44EC1A5
:1021D000D1014C91442309F4F2C02B31310529F48B
:1021E000F6018081882309F4EAC0F801EA5CFC4F1B
:1021F000808191810196918380836CE070E00E94E0
:102200002714892B09F0DBC02B31310529F0C901D6
:102210008E579109029710F4D6011C92F701608144
:102220007181C80141E050E0FC01E60FF71F3B97C8
:10223000A081FC01EE5AFC4FA0834F5F5F4F0196D7
:102240004C30510589F7F801E35AFC4F2083C8014F
:102250000E94AE0DD7018D909C90B3E08B1A91082F
:10226000F701918280825801612C712CF501EE5AA0
:10227000FC4F2081F501ED5AFC4F3081F501EC5AFD
:10228000FC4F9081632F822F2F83388799870E947C
:10229000F707AD81BE818C93998589272F81388579
:1022A000882309F44FC0982F9F70998382958F706F
:1022B0008A83FE01319680E090E041915FEF540FF8
:1022C0005230D8F14430C9F14830B9F14330E9F027
:1022D000453009F4C9C0463041F0473071F049300B
:1022E00071F050E04A3069F002C054E00FC04B304A
:1022F00051F04C3059F450E809C058E007C050E1A3
:1023000005C050E203C050E401C051E081309105A6
:1023100009F0A8C02527442381F0AB81BC814D91F1
:102320005D916D917C9113974F5F5F4F6F4F7F4F22
:102330004D935D936D937C93139701968230910535
:1023400009F0BBCFF20140815181FA01E227FF275A
:10235000EE0FFF1FE851FF4F85919491452F5527B0
:1023600084279527FC01E327FF27EE0FFF1FE85185
:10237000FF4F45915491892F992784279527D201A2
:102380008D939C93C30163E070E00E943B14660F41
:10239000771F680D791D600F711FFB01389720832F
:1023A000FB0137973083B3E06B0E711CE3E0AE0E98
:1023B000B11CFCE06F16710409F058CFFCCED601B9
:1023C0008C91811136C02E37310531F5F7018081AE
:1023D00091810C9748F0D2018D919C91883B904F50
:1023E00019F4C8010E94460781E0F10180838FEF54
:1023F0009FEFD2018D939C93F70111821082F80117
:10240000EA5CFC4F11821082AB81BC811D921D924F
:102410001D921C921397CFCE2F37310519F4F1017D
:102420001082C9CE2B31310521F481E0D6018C9385
:10243000C2CE4423A1F0F701808191818033F3E083
:102440009F0758F4AC014F5F5F4FD7014D935C93EA
:10245000F801E80FF91F208302C0F1011082D601B4
:102460001C92A9CE352757CF52E050CF29960FB6F0
:10247000F894DEBF0FBECDBFDF91CF911F910F91BA
:10248000FF90EF90DF90CF90BF90AF909F908F9094
:102490007F906F905F904F903F902F900895909312
:1024A0007F0880937E085093670840936608709376
:1024B0008208609381080895EF92FF920F931F9313
:1024C000CF93DF93EC01609166087091670880EC10
:1024D00090E00E940D15609166087091670880E099
:1024E00090E00E940D158E017E018CECE81A8CEFB5
:1024F000F80AF70180819181609166087091670800
:1025000098012C1B3D0B2817390708F5F80181911C
:102510008F01803C59F48BED90E00E940D15609185
:102520006608709167088CED90E00EC08B3D59F401
:102530008BED90E00E940D15609166087091670820
:102540008DED90E001C090E00E940D15D2CF80EC9F
:1025500090E0DF91CF911F910F91FF90EF900C943D
:102560000D158F929F92AF92BF92CF92DF92EF9212
:10257000FF920F931F93CF93DF93EC017B016A01CE
:10258000E0918108F09182088189811144C00E9404
:10259000BF1490910001891788F4A601B701CE01FC
:1025A000DF91CF911F910F91FF90EF90DF90CF902F
:1025B000BF90AF909F908F900C94A80D8FB7F89418
:1025C0008090620890906308A0906408B0906508BD
:1025D0008FBF209101013091020140910301509180
:1025E0000401AAE0B0E00E941C144FB7F8940091D7
:1025F00062081091630820916408309165084FBF0C
:10260000081919092A093B09061717072807390766
:102610000CF0B6CFEACFE0918108F0918208818971
:10262000882309F4ADCF80917E0890917F080E94A5
:10263000A310E0918108F0918208E853FF4F808158
:102640009181892B41F311821082DF91CF911F91EB
:102650000F91FF90EF90DF90CF90BF90AF909F9041
:102660008F900895882399F04091880850918908A7
:1026700066E171E080917E0890917F080E94B1121E
:10268000109283081092890810928808089580910A
:1026900083088823D9F02FB7F8948091620890912D
:1026A0006308A0916408B09165082FBF4091840829
:1026B000509185086091860870918708841B950B5E
:1026C000A60BB70BC397A105B10574F60895282F83
:1026D000809183088823A1F0203C01F580910D01B1
:1026E000811111C010928308409188085091890887
:1026F00066E171E080917E0890917F080C94B112A0
:10270000203C09F079C081E0809383088EEF8093AC
:102710000D01109289081092880808958091880808
:1027200090918908843233E0930708F065C03091B6
:102730000D01009731F43E3F21F42F7020930D01DD
:10274000089531111FC02B3D21F481E08093800852
:10275000089530918008332349F02C3D21F02D3D20
:1027600019F42BED01C020EC10928008AC014F5FF2
:102770005F4F5093890840938808FC01EA5EFE4F42
:1027800020830895313071F430E0AAE0B0E00E9477
:102790000D146093090170930A0180930B019093CB
:1027A0000C010895343089F43AE0239FC0011124CC
:1027B000AA2797FDA095BA2F809305019093060153
:1027C000A0930701B09308010895333089F43AE0EB
:1027D000239FC0011124AA2797FDA095BA2F8093AB
:1027E000010190930201A0930301B09304010895A5
:1027F000323011F42093000108950E9495018AE37C
:1028000094E00E94A31080E00E9412028823B9F392
:102810000E941C020E946713F2CFA29FB001B39FD7
:10282000C001A39F700D811D1124911DB29F700DD9
:10283000811D1124911D08950E940D14A59F900DD6
:10284000B49F900DA49F800D911D11240895AA1B83
:10285000BB1B51E107C0AA1FBB1FA617B70710F08B
:10286000A61BB70B881F991F5A95A9F780959095BD
:10287000BC01CD01089597FB072E16F4009407D0F4
:1028800077FD09D00E94271407FC05D03EF49095EF
:1028900081959F4F0895709561957F4F0895A1E2AE
:1028A0001A2EAA1BBB1BFD010DC0AA1FBB1FEE1FCA
:1028B000FF1FA217B307E407F50720F0A21BB30B15
:1028C000E40BF50B661F771F881F991F1A9469F791
:1028D00060957095809590959B01AC01BD01CF01ED
:1028E00008958F929F92AF92BF92CF92DF92EF9214
:1028F000FF92CF93DF93EC01688179818A819B817C
:10290000611571058105910521F464E279ED8BE58E
:1029100097E02DE133EF41E050E00E944715490177
:102920005A019B01AC01A7EAB1E40E941C146B019F
:102930007C01ACEEB4EFA50194010E944215C60ED5
:10294000D71EE81EF91EF7FE06C081E0C81AD1089E
:10295000E10880E8F80AC882D982EA82FB82C601CF
:102960009F77DF91CF91FF90EF90DF90CF90BF9056
:10297000AF909F908F9008950E94711408958EE0FB
:1029800091E00E9471140895A0E0B0E080930E01E0
:1029900090930F01A0931001B09311010895CF936C
:1029A000DF93EC012B8120FF33C026FF0AC02F7B71
:1029B0002B838E819F8101969F838E838A8190E0F5
:1029C00029C022FF0FC0E881F9818081992787FD06
:1029D0009095009719F420622B831AC03196F983E1
:1029E000E8830EC0EA85FB85099597FF09C02B8116
:1029F000019611F480E101C080E2822B8B8308C034
:102A00002E813F812F5F3F4F3F832E83992702C046
:102A10008FEF9FEFDF91CF9108950F931F93CF9387
:102A2000DF93182F092FEB018B8181FD03C08FEFFE
:102A30009FEF20C082FF10C04E815F812C813D81BD
:102A4000421753077CF4E881F9819F012F5F3F4FC4
:102A500039832883108306C0E885F985812F09957D
:102A6000892B29F72E813F812F5F3F4F3F832E8394
:102A7000812F902FDF91CF911F910F910895B7FF74
:102A80000C941C140E941C14821B930B0895052E99
:102A900097FB1EF400940E945E1557FD07D00E941C
:102AA0004F1407FC03D04EF40C945E1550954095DE
:102AB000309521953F4F4F4F5F4F089590958095EA
:102AC000709561957F4F8F4F9F4F0895F894FFCF7A
:102AD000FFC80000001900000096000000FE010081
:022AE0000000F4
:00000001FF
